:040000008A011C282D
:100008000C102618092826140A282610261C0D2844
:100018000D280900FF3E031D0E280800A40024082F
:10002800003C03181B28FF300E20A40313280800E7
:100038008316810181178312840185018B01FF30AA
:100048009900900185308400003080008F3083163D
:10005800810083128301101080308F008E018B0184
:100068008C308400013080008C010B178B170E3008
:10007800900010140730990085100511630042287C
:02400E0094011B
:00000001FF
